:02000000002AD4
:10000800A700030EA8008312031310100C1024304D
:100018008E022508031C250F8F021014A60A280E2D
:100028008300A70E270E09008A0182002F3441346D
:10003800353458340D3400342F3456343134503478
:1000480000342F344C3431344C340D3400342F34D4
:100058004C34313455340D3400342F344D3431346C
:10006800543431343134203400342F344D34313465
:100078005A340D3400342F344D343134543432343E
:100088003434203400342F344D343134543434343F
:100098003534203444345234203420344C345234EF
:1000A80020342034423452342034203453344834F9
:1000B8000D3400342F344D34313454343134323427
:1000C8003034203444344F344F34523420340034E4
:1000D8004F34503445344E342034203400344334C3
:1000E8004C344F3453344534443400342F344D3475
:1000F8003134543431343434303420345734413486
:10010800543445345234203400344F344E3420347F
:1001180000344F344634463400342F3455343134A7
:10012800433431340D3400342F34563431345034A0
:080138004A344A340D3400344E
:100200008A010A147808F80A82002F34083400346E
:1002100043340B34003431340E3400345634582A0D
:100220005A34972A5434992A4534652A26345B2A4D
:10023000533430345234483448345A344C346434AF
:10024000503456344634363447342C345734ED2A3F
:100250000D344D2A003400343134B02A00340034D7
:100260004134B72A5034B52A0034003431343C3498
:1002700032344234003400344134CF2A4234D22A5A
:10028000003400344134D52A4234D82A00340034B2
:1002900031344C340034003453345034003400349E
:1002A0003034FE2A3134042B003400344334FB2A2A
:1002B0000034003431345E340034003453340A2BBB
:1002C0005634272B003400344C34022B5534082B81
:0402D00000340034C2
:1004000083163F30850004308700003090000030B4
:10041000810091010C148312073099003130900053
:100420002430A400F430A500B401B50187150716E7
:10043000871607148714FA30712387110712871261
:1004400007108710A901AA01AB01AC01A301A20109
:10045000A101A601CD01CE010B178B176400682204
:10046000341E332A9B22071D362A2E2A09240530E2
:10047000F8002E24CC000021003A0319472A4C062C
:100480000319442AF80A3B2A0021F800392A0021DE
:10049000003A031D2E2A3F30C323FC2350222E2A6C
:1004A0000D30C32B50220E30382A2E30C323522A4F
:1004B00082305723522A4B085723522A522A871533
:1004C000053071238711A01208001A30B8232E2A94
:1004D0008B132608F63E03186F2A8B170800A60018
:1004E0008B17A10AA01621083C3A031D08003416F8
:1004F000A101A20A22083C3A031D0800A201A30A96
:1005000023080C3A0319AD0A23080D3A031D08000D
:10051000A301A30A3930B7239630AA234730B72363
:100520003C30AA239B223C30AA23DB2208008A22EB
:100530002E2A9B222E2A3412323071233130B823D6
:10054000230854233A30C323220851232030C323E5
:1005500041302D185030C3234D30C32350220800A2
:100560009130B7239830B7232E2A2D14B82A2D1096
:100570003B23A3003B23A200A101A6019B222E2A1C
:100580003230712307194D2A871587168714FA30E0
:100590007123871187128710FA307123C02A3B23F9
:1005A000A900DB2A3B23AA00DB2A3B23AB00DB2A82
:1005B0003B23AC00DB2A5022323071233F30B8237A
:1005C0002A08E9222908E9222C08E9222B08E92235
:1005D0004D2A57232030C3230800323071232E24A4
:1005E000CC0087104C1887147A30B82389304C1C03
:1005F0008D30B8234D2A071420154D2AC830712399
:100600002530B72387164D2AC83071232B30B723E6
:1006100087124D2A2E240339B9008711391C132B58
:10062000A01587152823B91C1A2B0716201E1C2B72
:100630001D231C2B071220164D2AA01D202B262B14
:10064000201D262B03302B2304302B234D2A2E2A4A
:1006500000302B230800B1002030B8233108413E80
:10066000C3230D30C3230800FF30BC07031CBD07A4
:100670003D083C040800C2012E24B7003030B70208
:10068000031C4F2B0A30370203184F2B0310C20DE7
:100690004208C20DC20DC2073708C2073C2B4208F0
:1006A0000800B415AE005D2BB411AE005D2BB41183
:1006B0005A2BB415AE00643061230A306123B4159F
:1006C0000130AF003030BE002F08AE02031C6B2B90
:1006D000BE0AB415652BAE073E08B41D2030C323F7
:1006E0000800F6008023F60B722B08000130812BE6
:1006F0000230812B0530812B0A30812B3230812B47
:100700006430F5000000000000000E30F400F40B2F
:10071000872BF50B822B08009D23B70033060319A6
:10072000932B0A30B2003708B300B20B08003A0628
:100730003705BB043708BA000800B701851C371419
:10074000051DB714851E3715051EB715051C371670
:1007500037080800B412C700C600C500071DB4164C
:10076000C50BAE2BC60BAD2BC70BAC2B0800000086
:10077000C8004808C80A1820B700003A0319080042
:100780003708C323B92BB7004F304D07CD0A84007B
:10079000370880000D3A031D0800CD01E02B03301F
:1007A000C400D923341B0800C8307123C40BD12BDB
:1007B0000800E0234F082F3A0319072C34170800CC
:1007C0004F308400E42BF823B001071DE32B7A237C
:1007D000B00BE52B071DE32B8316071183120008CE
:1007E00036240008840A0D3A031DEF2BCD010800C2
:1007F000FC233F39013E812B7108F2077208F30791
:100800000310F30C0318F3177308F1070800B4176B
:100810000A2CB4133413CE010030C6006430C50076
:100820007C235524B418C02A34181D2CC50B102C59
:10083000B41B0800C60B102C0800B7004E080F3A76
:1008400003192E2A5F304E07CE0A84003708800035
:100850000D3A031D0C2C3417CE0108005F304E07F3
:10086000CE0A840000080800CE030800C20002304F
:10087000712383160711831204304D2402304D2456
:100880000830BC000130C20D031803304D24BC0BEE
:10089000422C8316071583120800B7007C2307112A
:1008A0007C23B70B502C07150800B410341007191F
:1008B00008006D246D24CB000830BC00C2016D24FB
:1008C00003196B2CB7004B08B702C20DBC0B5F2C91
:1008D000420834140800B4140800B701B70A031919
:1008E00008000A30F400F40B732C07196E2CB701C2
:1008F000B70A031908000A30F400F40B7D2C3708FE
:06090000071D782C080021
:02400E00E200CE
:00000001FF
